:020000040000FA
:020000009E2838
:0800080009009801831603139F
:1000100098010C30990024309800C0308B008C1669
:10002000831203138030980008004130322054308E
:1000300032202B30322049303220503032205230A2
:1000400032203D30322031303220393032203230CF
:10005000322030303220303032200D3032200A3021
:10006000322008000C1E3228990008000D30322082
:100070000A30322008002C30322008004130322073
:10008000543032202B303220433032204D30322059
:1000900053303220533032203D30322008003E2091
:1000A000313032203B20362008003E2032303220D2
:1000B0003B20362008003E20333032203B203620C3
:1000C00008003E20343032203B20362008003E20FD
:1000D000353032203B20362008003E20363032209A
:1000E0003B2036200800413032205430322044304A
:1000F00032203E303220533032204D3032203130E9
:1001000032203B3032200D30322008004130322086
:1001100054303220483032200D3032200800640044
:10012000861F9828431D08006D20C3104311080046
:10013000C3180800C3146720431508008B138312EB
:10014000850107309F0000308316850083128601E9
:10015000FB30831686008312C901861EB52A061E4F
:10016000572A831679309B001C14831203101A1827
:100170002E299A18EC28CA288312C3014922492241
:1001800005118511C910003083169A0079309B0043
:10019000A5223B228312061E572A861EB52A6621F7
:1001A000C91CCA28D32883120520152002308316C3
:1001B0009A0079309B00A5228312C91085153B2235
:1001C0008511061FE7286621C91CE128BC280510F7
:1001D0008510851549220511831285155520640067
:1001E0008F20FF306200C910061BFC286621C91849
:1001F000FA28EF286120BC284F206400FF306200FD
:100200000130BD0005158511F121C91C0829BC2844
:100210008515F121C91C0D29BC28BC0B0229BD0B79
:1002200002290511061B152928295B208F20851519
:1002300005153B223B22851105116621C91C212988
:10024000BC283B223B223B223B22061B16292829A5
:10025000013083169A0079309B00A5228312640036
:10026000FF30620085150511061F3B293729F12152
:10027000C91C3B29BC288511061F43293F29F121B0
:10028000C91C2E29BC28552064008F20FF30620035
:10029000061BFC28F121C91C5229C91C5229C91C62
:1002A0005229BC2885116400FF306200061BFC281F
:1002B000F121C91C5C29BC28F121C91C6029BC287A
:1002C000F121C91C6429BC28851544293722102234
:1002D0003122022237222522061C7B291E22061CDF
:1002E00072297B291022061C7B297D219C21D12289
:1002F000491D7B29BF21312208003330B600083068
:10030000BA003122361C852987291E229629000031
:10031000000000000000000037221E229729000084
:100320000000000000000000000081293722B60C08
:10033000BA0B8F291E2208000310203084000830D9
:10034000BA0083169B018312AB2135088000840A12
:10035000BA0BA42908000830BB00312200000000BD
:100360000000000037222522061CB829B517B9293C
:10037000B513B50C1E22BB0BAD29B50D0800C80185
:10038000CE290830C80778304802031DCE29C9108D
:100390003122102205153B2205110800203084006F
:1003A000480883169B0083120830BA0083161C1479
:1003B0008312031083161A0883120002031DC12939
:1003C000840A83169B0A8312BA0BD6290030A00038
:1003D000A100A200A300A400A500A600A700C914C4
:1003E00008006400FF306200B001B101A030B2002B
:1003F000B00BFB29FF296621C91CFF290800B20B9D
:10040000F82908000630B100B000B00B052AB10B86
:10041000042A0730B100B000B00B0C2AB10B0B2A34
:100420000430B100B000B00B132AB10B122A053012
:10043000B100B000B00B1A2AB10B192A0430B10078
:10044000B000B00B212AB10B202A000000000000F0
:10045000000000000000000000006400FF306200A7
:100460000800061083160610831206100800831673
:10047000061483120800B001B1010530B200B00BC0
:100480003F2AB10B3F2A6400FF306200B20B3F2AC3
:100490000800B001B1010130B200B00B4D2A640078
:1004A000FF306200B10B4D2AB20B4D2A0800BC018F
:1004B000BD01061E572A5C2ABD0B652ABC0B652AA6
:1004C0000515492205118511CA28851549113722BC
:1004D0001E223122022237222522061C5C2A1E22DD
:1004E000061C732A5C2A1022061C5C2A7D219C2192
:1004F000D122491D5C2A7C2A831678309B001C146B
:100500001A02031D842A9A0183161A089B0083127B
:100510000830BA0020308400000883169A00A52213
:100520008312840A83169B0A8312BA0B8C2A8316C1
:100530001B089A0078309B008312A52205154922DA
:100540000511851149228515572A83161C151C1083
:100550008B1355309D00AA309D009C141C118312F2
:100560008C1FB02A8C13831208008312003083166C
:100570009B0008309A0083127830BA00A5228316B7
:100580009B0A8312BA0BBE2A05158515492205114F
:1005900085113B22783083169B0000309A00A522FB
:1005A000572ABE0149112008C100F0222108C100CC
:1005B000F0222208C100F0222308C100F022240802
:1005C000C100F0222508C100F0222608C100F02257
:1005D0002708C100F02200303E0203194915080027
:1005E0000830C00041083E06BF003F0C3E0803181B
:1005F000183ABF003F0CBE000310C10C4108C00BED
:04060000F32A0800D1
:02400E000D3F64
:00000001FF
